:020000040800F2
:1000000000100020C5170008A9020008AD02000872
:1000100000000000000000000000000000000000E0
:10002000000000000000000000000000B102000815
:100030000000000000000000B5020008B90200083E
:1000400015180008151800081518000815180008DC
:1000500015180008151800081518000815180008CC
:1000600000000000151800081518000815180008F1
:1000700015180008151800081518000800000000E1
:1000800015180008151800080000000015180008D1
:100090001518000815180008BD02000815180008FA
:1000A0001518000815180008151800083103000875
:1000B000151800080000000000000000000000000B
:0C00C000151800080000000015180008CA
:1000CC0003B47146490840004900095E49008E445A
:1000DC0003BC7047844608006146FFE71FB503F078
:1000EC00C9FA002801D40021C8421FBD10B503F085
:1000FC0057FA4042013010BD10B503F0BBFA00288E
:10010C0001DB002010BD012010BDC04610B503F06E
:10011C00B1FA002801DD002010BD012010BDC04641
:10012C0010B503F065FA002801DC002010BD012099
:10013C0010BDC04610B503F05BFA002801DA0020B0
:10014C0010BD012010BDC0461C2101231B04984288
:10015C0001D3000C10391B0A984201D3000A08394C
:10016C001B09984201D30009043902A2105C401803
:10017C007047C046040302020101010100000000A7
:10018C000000000040F2640040F26403C2F2000080
:10019C00C2F2000310B5834205D040F20003C0F256
:1001AC00000303B1984710BD40F2640040F26403B1
:1001BC00C2F20000C2F200031B1A9A10D90F891860
:1001CC00491010B529B140F20003C0F2000303B18D
:1001DC00984710BD10B540F26404C2F200042378B5
:1001EC0073B9FFF7CFFF40F20003C0F200032BB14D
:1001FC0043F20070C0F6000000E000BF0123237042
:10020C0010BDC04640F20003C0F2000310B54BB164
:10021C0040F2680143F20070C2F20001C0F6000027
:10022C0000E000BFFFF7C0FF10BDC04640F2140352
:10023C00C2F200031B68002110B5986801F0C2FBE4
:10024C0000F0BCF800F0B0F900F042FB00F084FBC9
:10025C0000F020F900F0FCFC632000F0F7F800F04F
:10026C00F7FDF9E770B5161E15DD0C008D1843F679
:10027C0000002178C4F2010001F04CFA43F60000B2
:10028C0040F20771C4F2010001F050FA0028F5D0D9
:10029C000134AC42EBD1300070BDC046FEE7C04625
:1002AC00FEE7C046FEE7C046FEE7C0467047C046C4
:1002BC0044F6000010B50121C4F2010001F0B4F9BC
:1002CC00012800D010BD44F6000040F2A104012129
:1002DC00C4F20100C2F2000401F0B2F9237893B920
:1002EC0090208021C005012200F04EFE44F6000053
:1002FC0040F22031C4F2010001F090F923785A4207
:10030C0053412370DEE7902000228021C00500F0CD
:10031C003BFE44F6000044F60031C4F2010001F04B
:10032C007DF9EBE7052143F6000010B5C0F205712D
:10033C00C4F2010001F010FA50B9042143F6000098
:10034C00C0F20471C4F2010001F006FAF0B910BD5C
:10035C00052143F60000C0F20571C4F2010001F062
:10036C0015FA43F60000C4F2010001F0D9F940F28D
:10037C00A003C2F200031A781E2ADED8511C197091
:10038C0040F28003C2F200039854D6E7042143F6EE
:10039C000000C0F20471C4F2010040F2A00401F0AC
:1003AC00F5F940F28000C2F200042178C2F200009C
:1003BC0000F0C6F900232370C9E7C046052010B52C
:1003CC00404200F06DFE40F20403C2F200031868D4
:1003DC0003F0A6F842F20041C4F6F42102F06AFCE4
:1003EC0040F2A8030021C2F2000318601868C4F29E
:1003FC007A4102F071FD40F2A403C2F200031860CE
:10040C0010BDC04640F2A803C2F2000310B51C6830
:10041C0003F086F8211C02F05FFD02F033FC4EF273
:10042C00100200230121CEF20002506093600133D0
:10043C001360C0F2010113680B40012BFBD00121AA
:10044C0013688B4313600023936010BD40F2A40328
:10045C00C2F2000310B51C6803F062F8211C02F014
:10046C003BFD02F00FFC4EF2100200230121CEF2F4
:10047C0000025060936001331360C0F201011368F5
:10048C000B40012BFBD0012113688B43136000231D
:10049C00936010BD40F2102310B582B001AC220065
:1004AC0023801421562000F07FFB41F600632200CC
:1004BC0023801021562000F077FB44F205632200C4
:1004CC0023800821562000F06FFB0023220023809C
:1004DC001921562000F068FB9023220023801E2156
:1004EC00562000F061FB40F60243220023801B21C2
:1004FC00562000F059FB40F2161322001A212380DB
:10050C00562000F051FB02B010BDC04670B504007F
:10051C00002382B001AD01002A00562001342B804B
:10052C0000F068FB2A005620E1B22E8800F062FB36
:10053C00288876BA40BA360480B2304303011033AF
:10054C0013D0030E00280DDB5A0608D49A0603D4E8
:10055C00DB060DD402B070BD80208005FAE7802048
:10056C00C005F7E780200006F4E7F0200006F1E76D
:10057C0080204005EEE7C046002310B582B001ACE8
:10058C00220000219220238000F034FB2278637833
:10059C0012011B0913435801C01A8000C0188300B4
:1005AC00C01802B010BDC04610B5902440F21150D6
:1005BC00E40500F083FD40F20E6000F07FFD2000AA
:1005CC000C22012100F0EEFC20000C230122022160
:1005DC0000F08AFC20000C230122002100F0B0FC6A
:1005EC00200002230022012100F07EFC02232000C7
:1005FC000322002100F0A4FC200043F60004012299
:10060C00C4F20104022100F0BFFC200001F01CF830
:10061C00E1212000490201F037F82000042101F00B
:10062C0071F80821200001F065F8200001F05CF859
:10063C0000211B2000F0EEFC2000052101F080F8C9
:10064C000421200001F07CF810BDC04630B500201C
:10065C0085B0FFF75BFF40F2AC0440F20005C2F23C
:10066C00000400BA20600B20C2F200052A8802ABFD
:10067C001A80AA7821009A706844042201F0DBFBEE
:10068C0043F23070AB786A782978C0F6000001F03C
:10069C007FF9E078A37821786278009043F2447077
:1006AC00C0F6000001F074F909230F2100206B44FF
:1006BC0069441A7801338018C0B28B42F9D101F029
:1006CC0077F905B030BDC04630B585B0FFF754FFA3
:1006DC0040F2AC0440F20005C2F2000400BA206003
:1006EC000B20C2F200052A8802AB1A80AA782100DE
:1006FC009A706844042201F09EFB43F23070AB7890
:10070C006A782978C0F6000001F042F9E078A37805
:10071C0021786278009043F24470C0F6000001F03A
:10072C0037F909230F2100206B4469441A780133EF
:10073C008018C0B28B42F9D101F03AF905B030BD46
:10074C00F0B543788678033B5A1E934102789B00A0
:10075C00D53A541EA24152001343B21E541EA2415C
:10076C00D7001F43FF2319404D1E435D87B09C46A5
:10077C00022900D891E00023421C4519147801325B
:10078C001B19DBB29542F9D101229C4504D10436E8
:10079C00761A731E9E41F2B23A43082A13D893007C
:1007AC004A4AD3589F46402343F250700393323346
:1007BC00029301930D3B0093F422B521623BC0F6EA
:1007CC00000001F0E5F807B0F0BD43F2387105AC5C
:1007DC000379C278C0F60001200001F0AFF923784C
:1007EC004D2B02D16378312B59D023784D2B3AD134
:1007FC006378322B37D1A378ABBBFFF765FFE2E709
:10080C003D2343F2507003933533029301930D3B18
:10081C000093F122B521623BC0F6000001F0B8F85C
:10082C00D1E73E2343F25070039334330293019388
:10083C000D3B0093F222B521623BC0F6000001F0A3
:10084C00A7F8C0E73F2343F250700393333302936E
:10085C0001930D3B0093F322B521623BC0F60000DF
:10086C0001F096F8AFE723784D2B1ED16378332B2C
:10087C001BD1A378CBB943F24070CC330293613BCC
:10088C0001930433F122B5210093C0F600006D3BB7
:10089C0001F07EF800F0EEF995E7002374E7A378F9
:1008AC00002BA2D1FFF7D2FE8DE73C2343F2507010
:1008BC0003933633029301930D3B0093F022B52141
:1008CC00623BC0F6000001F063F87CE7603700087B
:1008DC0010B5902484B0E40540F2115000F0EEFB0A
:1008EC00200080230022012100F0FEFA802320004A
:1008FC000322002100F024FB200044F60004012216
:10090C00802100F041FBC4F2010440F2126000F0BF
:10091C00D5FB200000F096FD684600F0FFFD42F28A
:10092C000F73029341F61F43009300236946200086
:10093C00019300F0FBFD200000F06AFE0121200075
:10094C0000F06EFE200000F05DFE0221162000F08B
:10095C0061FB04B010BDC04610B541F20044C4F6B2
:10096C00000440F2165000F0A9FB200002230122E3
:10097C00012100F0B9FA200002230322012100F02A
:10098C00DFFA200001230122012100F0ADFA01233E
:10099C0003222000012100F0D3FA2000022100F0F4
:1009AC00EFFA0121200000F0EBFA10BD10B541F276
:1009BC000044C4F600042000012100F0E1FA0221F9
:1009CC00200000F0DDFA1420FFF71CFD01212000AF
:1009DC0000F0D8FA1420FFF715FD0221200000F0DA
:1009EC00D1FA10BD10B541F20044C4F60004200049
:1009FC00022100F0C7FA0121200000F0C3FA1420F4
:100A0C00FFF700FD0221200000F0BAFA1420FFF7D6
:100A1C00F9FC0121200000F0B3FA10BD10B541F231
:100A2C000044C4F600040121200000F0ABFA1420AD
:100A3C00FFF7E8FC0221200000F0A2FA1420FFF7D7
:100A4C00E1FC0221200000F09DFA1420FFF7DAFCF3
:100A5C000121200000F094FA10BDC04610B541F2FF
:100A6C000044C4F600040121200000F089FA14208F
:100A7C00FFF7C8FC0221200000F082FA1420FFF7D7
:100A8C00C1FC0221200000F07DFA1420FFF7BAFC13
:100A9C000121200000F074FA10BDC04670B541F27F
:100AAC000045C4F600052800012100F069FA142065
:100ABC00FFF7A8FC2800022100F062FA1420FFF7CF
:100ACC00A1FC2800012100F065FA040063425C419E
:100ADC002800022100F056FAE0B270BD70B5040097
:100AEC0008251CE000F04EFA1420FFF78BFC41F2B5
:100AFC0000400221C4F6000000F042FA1420FFF777
:100B0C0081FC41F200400221C4F6000000F03AFAE8
:100B1C0064001420013DFFF775FCE4B255B141F2BD
:100B2C00004063B20121C4F60000002BDADA00F0B9
:100B3C0027FAD9E770BDC046F8B5070041F200406E
:100B4C000121C4F6000000F01BFA08250024012640
:100B5C0041F200400221C4F6000000F011FA14200A
:100B6C00FFF750FC41F2004064000121C4F6000084
:100B7C00E4B200F00FFA08B13443E4B241F20040A1
:100B8C000221C4F6000000F0FDF9013D1420FFF72E
:100B9C0039FC002DDCD11FB1FFF740FF2000F8BD60
:100BAC00FFF75CFFFAE7C04670B504000E001500B5
:100BBC00FFF7FCFE2000FFF791FFFFF76FFFA0B1DE
:100BCC003000FFF78BFFFFF769FF70B12878FFF754
:100BDC0085FFFFF763FF40B16878FFF77FFFFFF7F2
:100BEC005DFFFFF7FFFE012002E0FFF7FBFE002098
:100BFC0070BDC04670B504000D001600FFF7D6FEA0
:100C0C002000FFF76BFFFFF749FFE8B12800FFF763
:100C1C0065FFFFF743FFB8B1FFF7C8FE0120204383
:100C2C00FFF75CFFFFF73AFF70B11420FFF7EAFB08
:100C3C000120FFF781FF30700020FFF77DFF7070FF
:100C4C00FFF7D0FE012002E0FFF7CCFE002070BDC4
:100C5C0010B540F6001000F0FFFA40F6001000F05E
:100C6C005DFA042140F2712000F0FAF800F0E8F887
:100C7C0010BDC04643F2000345F2555210B5C4F204
:100C8C00000300211A60322000F0EAF800F0E0F8CE
:100C9C0010BDC04641F20002012110B5C4F202029F
:100CAC00136882B00B431360013113681942FCD0F6
:100CBC0041F204038021C4F202031A680A431A6049
:100CCC0000230193019B7F2B05D8019B01330193DA
:100CDC00019B7F2BF9D941F204039021C4F202034A
:100CEC001A680A431A6000230193019B7F2B05D8D5
:100CFC00019B01330193019B7F2BF9D941F2040332
:100D0C000321C4F202031A684FF6FF708A4341F2C2
:100D1C0000011A60C4F202010A68CFF6F2600240C8
:100D2C000C200A601A68C0F6FF0002404FF6FF70F4
:100D3C001A601A68C7F2C27002401A6041F22C03A2
:100D4C000F20C4F202031A6882431A6041F2300386
:100D5C00C4F202031A68384802401A601A6837480D
:100D6C0002401A601A680120520052081A6041F2BF
:100D7C003403C4F202031A6882431A6041F2080376
:100D8C000022C4F202031A600B6803430B600130AB
:100D9C0040F2005301E0013B13B10A681042FAD053
:100DAC0041F200020221C4F202021368194241D03E
:100DBC0042F200000724C4F202000368A3430B4371
:100DCC00036041F204034FF6FF70C4F2020319688A
:100DDC00CFF2C27019601968196019681960196826
:100DEC000140196000211868C0F604010143196024
:100DFC00802311685B040B43802113608904136802
:100E0C000B42FCD041F204020321C4F2020213682B
:100E1C008B431360136801390B4313600A31136859
:100E2C000B40082BFBD180200021000500F02AF993
:100E3C0002B010BDFEE7C046FCFEFFFFFFFFFEFF49
:100E4C0043F200034CF6CC42C4F200031A60704724
:100E5C0043F200034AF6AA22C4F200031A60704758
:100E6C0043F2000345F25552C4F2000330B543F28D
:100E7C000C041A604FF6FF720125C0F20F02C4F287
:100E8C0000042368013A2B4032B3002BF9D143F212
:100E9C000403C4F200034FF6FF72196043F20C0115
:100EAC000224C0F20F02C4F200010B68013A234085
:100EBC00B2B1002BF9D140F6FF7343F208020340A4
:100ECC00C4F20002136043F200034AF6AA22012086
:100EDC00C4F200031A6030BD002BD8D00020FAE712
:100EEC00002BE8D00020F6E7F0B54546DE46574625
:100EFC004E468C46904683461A000024012140F24F
:100F0C000309E0B50768C5680E00A64032420AD056
:100F1C004E46604663009E409840B74307434046A8
:100F2C009840B54305430134102CEDD15B461F604E
:100F3C00DD60F0BCBB46B246A946A046F0BDC0463B
:100F4C00F0B5012917D04168994341600021012671
:100F5C0040F2030C846835008D402B4206D0674666
:100F6C004D00AF40BC431700AF403C43013110294A
:100F7C00F1D18460F0BD416819434160E6E7C04699
:100F8C0081617047816270470AB1816170478162EB
:100F9C00FCE7C046036919400800431E9841C0B2E3
:100FAC007047C046F0B5CE464746036A89469C4614
:100FBC000126002340F20F0880B5456A34009C409E
:100FCC0022420AD047469C00A7406146B9430F0015
:100FDC004946A1400C003C43A4460133082BEDD1FB
:100FEC000024012740F20F083E009E40324205D0FB
:100FFC0046464946A640A140B5430D43013304344F
:10100C00102BF1D1634603624562C0BCB946B046B1
:10101C00F0BDC046FF22032330B514000340DB00B3
:10102C009C4089010A409A4043B2E443002B19DBEF
:10103C004EF20011CEF200018C4640F200358308CE
:10104C009B006344595921400A431F215A510122E4
:10105C0001408A404EF200114309CEF200019B0080
:10106C005A5030BD4EF600510F23CEF200018C4683
:10107C000340083B9B089B006344D9690C40144314
:10108C00DC61EEE74FF68073C1F6FF7319404EF644
:10109C0000530143CEF200039960BFF34F8F7047AA
:1010AC004EF21003CEF200031A68042803D0042178
:1010BC008A431A60704702431A60FBE741F200034F
:1010CC001F21C4F202039C46012301408B4010B542
:1010DC008209624414682343136010BD41F200037B
:1010EC001F21C4F202039C46012301408B4010B522
:1010FC008209624414682343136010BD41F200025C
:10110C001F21C4F202029446830908401E39814013
:10111C0063441A688A431A607047C04640F600035D
:10112C00984200D181E01AD8102868D018284ED0E7
:10113C0040F20053002831D141F200010230C4F2D8
:10114C00020101E0013B13B10A681042FAD041F2EE
:10115C000003C4F2020318688007C00F704740F602
:10116C00001398421CD040F60053984216D14FF60B
:10117C00FF7341F234010220C0F20F03C4F20201EA
:10118C0001E0013B13B10A681042FAD041F234037A
:10119C00C4F2020318688007C00FDFE70020DDE708
:1011AC004FF6FF7341F224010220C0F20F03C4F288
:1011BC00020101E0013B13B10A681042FAD041F27E
:1011CC002403C4F2020318688007C00FC6E74FF669
:1011DC00FF7341F200018020C0F20F03C4F2020140
:1011EC00800401E0013B13B10A680242FAD041F2DB
:1011FC000003C4F2020318688001C00FAEE741F28D
:10120C00000180204FF6FF73C4F20201800201E05E
:10121C00013B13B10A680242FAD041F20003C4F256
:10122C00020318688003C00F98E741F220010220E6
:10123C00084BC4F2020101E0013B13B10A681042F1
:10124C00FAD041F22003C4F2020318688007C00FE1
:10125C0084E7C046FFFFFF0341F200031F21C4F2E5
:10126C0002039C46012301408B4010B58209624465
:10127C0014682343136010BD43F21873F0B589B0A2
:10128C00C0F60003020004A81C000100E0CCE0C181
:10129C006D4624680C6019002C001031C0C9C0C404
:1012AC0021001033C0CBC0C141F204010C23C4F2A5
:1012BC0002010E683340082B22D041F20023C0F209
:1012CC007A0341F204061F00C4F2020631680906D3
:1012DC00090F415C0720CF403168090A01406D5C61
:1012EC003168C90A0840215C3800C840052A00D979
:1012FC00A3E0534992008A589746380009B0F0BDD4
:10130C000B6809689B021B0F090119D40F2B76D0AF
:10131C00023341F20401C4F202010968C90317D572
:10132C0041F22C01C4F202010E680F21314041F24E
:10133C0000260131C0F27A06B6FBF1F67343C0E722
:10134C0041F20401C4F2020109681133C903E7D464
:10135C005E01F61AB101891BC900CB181B02B0E75C
:10136C001800CBE741F230010322C4F202010C68F1
:10137C002242C3D00C6818001440012CBED00B685C
:10138C001340022B52D00B6841F200201340033B58
:10139C005A425341C0F27A005B421840AEE7380023
:1013AC00E840ABE741F23003C4F202031A68D205FD
:1013BC000ED4186849F68073C003C0F2D503C01769
:1013CC00184049F68073C0F2D5039C46604495E7FB
:1013DC0041F204020321C4F2020212681B68920B50
:1013EC000A40DB0F022A14D0032A0AD0012A15D096
:1013FC004008002B00D181E7B7FBF1F07EE710230A
:10140C0087E7C008002B00D178E70920B7FBF0F084
:10141C0074E773B90633B0FBF3F06FE78008002B69
:10142C0000D16BE70520B7FBF0F067E748F200004E
:10143C0064E70720B7FBF0F060E700205EE7C046EA
:10144C008437000842F60043C4F2010310B59842F9
:10145C0048D01AD841F20003C4F20003984253D08A
:10146C0042F20003C4F20003984232D040F200432F
:10147C00C4F20003984207D140F20140FFF72EFE60
:10148C0040F20140FFF73AFE10BD44F20043C4F2B3
:10149C00010398422FD044F60003C4F20103984292
:1014AC000ED044F20003C4F201039842ECD140F296
:1014BC001030FFF713FE40F21030FFF71FFEE3E78A
:1014CC0040F21230FFF70AFE40F21230FFF716FE20
:1014DC00DAE740F20840FFF701FE40F20840FFF760
:1014EC000DFED1E740F20B30FFF7F8FD40F20B3068
:1014FC00FFF704FEC8E740F21130FFF7EFFD40F2B2
:10150C001130FFF7FBFDBFE740F20440FFF7E6FDAB
:10151C0040F20440FFF7F2FDB6E7C0464FF6FF730A
:10152C008360002303604360037370470B8810B51E
:10153C00836242F60043C4F20103984228D040F281
:10154C000043C4F20003984222D08B68C36242F27B
:10155C000003C4F20003984249D044F20003C4F2E1
:10156C00010398420BD044F20043C4F201039842A9
:10157C0005D044F60003C4F20103984226D1036857
:10158C001F4A134003600268CB88134303601BE0BF
:10159C00702203689343036002684B881343036013
:1015AC0002688B88134303608B68C36242F6004366
:1015BC00C4F20103CA8898420DD10368104C234031
:1015CC0003600368134303600B7B036301224369CD
:1015DC001343436110BD40F20043C4F20003196889
:1015EC00074C2140196019680A431A60EEE703683A
:1015FC00034A134003600268CB8813430360E5E79A
:10160C00FFFCFFFF01220368134303607047C046D1
:10161C0080220368134303607047C046C162704761
:10162C00C3680B43C3607047C2680369194204D096
:10163C0011404B1E9941C8B270470020FCE7C046D0
:10164C00C94301617047C04644F20043C4F2000331
:10165C0010B598420FD043F60003C4F20103984230
:10166C0000D010BD40F20E30FFF738FD40F20E30C6
:10167C00FFF744FDF5E740F21140FFF72FFD40F274
:10168C001140FFF73BFDECE744F20043C4F20003CA
:10169C0070B504000D00984222D043F60003C4F24A
:1016AC00010300209C4217D023686A081B040BD549
:1016BC0043009B18B3FBF5F54FF6F0722B075B0F4D
:1016CC002A401343E36070BD8218B2FBF5F54FF668
:1016DC00FF732B40E360F6E70530FFF7CDFDE3E742
:1016EC000220FFF7C9FDDFE7012203681343036003
:1016FC007047C046082203689343036003680B439A
:10170C0003607047042203689343036003680B4330
:10171C000360704740F2FF130B4083627047C04672
:10172C00436A40F2FF1018407047C0461F228B09D5
:10173C001B181B680A40D340012018407047C04654
:10174C008B091F22181801230A40934010B5046816
:10175C002343036010BDC0460B049B0D8A0D121869
:10176C001B18012070B51F2406001B6815680A0C95
:10177C0022409640354206D00C40A04003405A1EF1
:10178C009341D8B270BD0020FCE7C04643F2094338
:10179C00C3F20F43994207D00123C902C90E8B40F3
:1017AC00026A134303627047D0300368014A134046
:1017BC000360F8E7FF7FFFFF0D488546002103E03B
:1017CC000C4B5B58435004310B480C4B42189A425B
:1017DC00F6D30B4A02E0002313600432094B9A4201
:1017EC00F9D3FFF757FA00F0FBFAFEF71FFDFEE7FF
:1017FC000010002054380008000000206400002075
:10180C006400002000020020FEE70000002310B559
:10181C00040003604360836081814366C28103617D
:10182C0043618361190008225C3000F08BFA0B4B8A
:10183C00246263620A4BA3620A4BE3620A4B236382
:10184C000A4B9C4205D00A4B9C4202D0094B9C424D
:10185C0003D12000583000F0EBFA10BD8D1B0008AE
:10186C00B51B0008ED1B0008191C0008B000002077
:10187C00180100208001002010B5034A03490448D8
:10188C0000F06AF810BDC04608000020812900084D
:10189C001800002041680B4B10B50400994201D090
:1018AC0001F068F8A168084B994202D0200001F0C1
:1018BC0061F8E168054B994202D0200001F05AF81A
:1018CC0010BDC046B000002018010020800100208F
:1018DC0010B5094B094A04211A6009480022FFF788
:1018EC0095FF012209210748FFF790FF02221221E0
:1018FC000548FFF78BFF10BDE80100208518000894
:10190C00B0000020180100208001002010B5024812
:10191C0000F08FFA10BDC046F101002010B502484E
:10192C0000F088FA10BDC046F101002010B504008B
:10193C00FFF7ECFF236A13B1FFF7F0FF10BD044B68
:10194C002362044B1B68002BF6D1FFF7C1FFF3E7B2
:10195C00A1180008E8010020F7B51400002600903B
:10196C000191A5686768013F04D52468002CF8D163
:10197C003000FEBDAB89012B08D90E22AB5E0133C2
:10198C0004D029000098019B984706436835EAE784
:10199C000FB407B5054904AB086804CB8168019303
:1019AC0000F0DCFC03B008BC04B0184714000020A5
:1019BC0010B5034B01001868826801F06BF810BD7C
:1019CC00140000204A424A4110B540F20043520034
:1019DC0000F002F810BD0000F0B51D00554B85B0AD
:1019EC001E6804000F00009226B1336A13B9300050
:1019FC00FFF79CFF009B022B05D0012B00D996E032
:101A0C00002D00DA93E0636EDB0705D4A3899B05F8
:101A1C0002D4A06D00F00DFA2100300000F0AAFFF6
:101A2C00616B41B123004433994202D0300000F085
:101A3C000BFA002363630023A3616360A3891B0675
:101A4C0003D53000216900F0FFF9A3893A4A13400D
:101A5C00A381009B022B60D003AB2100300002AAB3
:101A6C0000F0B0FFA3890343A3812DBB029D280086
:101A7C0000F032FA01950700002848D1029B01932F
:101A8C00AB423ED101256D420C22A35E02221A43C9
:101A9C00A2810022A2602200473222602261012230
:101AAC00616E6261114204D19B0502D4A06D00F0FD
:101ABC00C1F9280005B0F0BD002FD8D0336A13B996
:101ACC003000FFF733FF009B012B03D1A389009A51
:101ADC001A43A2810C22A35E0822190027602761F9
:101AEC006561114013421CD0DA0718D500226D42F3
:101AFC00A260A561626ED20701D49B0513D50025A7
:101B0C00D7E7019800F0E8F907000028BAD0802345
:101B1C00A289019D1343A381D0E70025B4E7A560FA
:101B2C00E8E7A160E6E7A06D00F084F9E7E701259E
:101B3C006D42BEE7140000205CF3FFFF0EB410B53D
:101B4C0000240C499DB01FAB0290069007910491A4
:101B5C0009480A4904CB0591006802A901931B941A
:101B6C0000F0D8FA029B1C701DB010BC08BC03B06E
:101B7C001847C046FFFFFF7F140000200802FFFF3C
:101B8C0070B50C000E25495F00F006F9002803DB48
:101B9C00636D1B18636570BDA389024A1340A38152
:101BAC00F9E7C046FFEFFFFFF8B51F008B89050072
:101BBC000C001600DB0505D50E23C95E002202239E
:101BCC0000F0D8F8A389054A28001340A3813200FD
:101BDC000E23E15E3B0000F0F1F8F8BDFFEFFFFFD4
:101BEC0070B50C000E25495F00F0C4F8A389421CA7
:101BFC0003D1054A1340A38170BD41F20002134387
:101C0C00A3816065F8E7C046FFEFFFFF10B50E2318
:101C1C00C95E00F09FF810BDF8B506000D00140069
:101C2C0018B1036A0BB9FFF781FEA369A360A389FE
:101C3C001B0701D5236943B92100300000F02AF8B5
:101C4C0018B101256D422800F8BD23692068EFB258
:101C5C00C01A6369EDB2834205DC2100300000F04C
:101C6C0089FE0028EDD1A3680130013BA3602368F5
:101C7C005A1C22601F706369834204D0A389DB075E
:101C8C00E1D50A2DDFD12100300000F073FE0028D1
:101C9C00D9D0D6E72A4B70B5050018680C0018B1DE
:101CAC00036A0BB9FFF742FE0C22A35E1A0722D47B
:101CBC00DA0607D409222A60402201201343A381AB
:101CCC00404237E05B0712D5616B41B123004433CE
:101CDC00994202D0280000F0B7F800236363242255
:101CEC00A3899343A38100236360236923600823A2
:101CFC00A2891343A38123695BB940F2802140F28E
:101D0C000022A3890B40934203D02100280000F04D
:101D1C0083FE0C22A35E01211A000A400B420AD05A
:101D2C000022A26062695242A261226900200AB9B3
:101D3C001A06C1D470BD990700D46269A260F4E799
:101D4C001400002003008218934200D170471970D0
:101D5C000133F9E7002370B5054D040008002B6032
:101D6C0000F050FF431C02D12B6803B1236070BDFF
:101D7C00EC01002070B50400080011001A000023CB
:101D8C00044D2B6000F05AFF431C02D12B6803B1A9
:101D9C00236070BDEC01002070B504000800110038
:101DAC001A000023044D2B6000F052FF431C02D19B
:101DBC002B6803B1236070BDEC01002070B50400EA
:101DCC00080011001A000023044D2B60FEF74AFA9C
:101DDC00431C02D12B6803B1236070BDEC010020C1
:101DEC0070B500250E4C0F4BE41AA410A54209D176
:101DFC00002501F07FFC0C4C0C4BE41AA410A542FE
:101E0C0007D170BD074AAB009B181B68984701357A
:101E1C00ECE7064AAB009B181B6898470135EEE7C8
:101E2C004C3800084C380008503800084C38000872
:101E3C00704770477047002310B59A4200D110BD0F
:101E4C00CC5CC4540133F8E770B505000C0079B1D3
:101E5C00043C2368002B00DAE418280000F0E8F8B2
:101E6C001C4A13682BB963601460280000F0E8F872
:101E7C0070BDA34208D9206821188B42F3D1196890
:101E8C005B6809182160EEE71A005B680BB1A3428E
:101E9C00FAD911685018A0420BD1206809185018B3
:101EAC0011608342E1D118685B684118116053607E
:101EBC00DBE7A04202D90C232B60D6E7206821185F
:101ECC008B4203D119685B68091821606360546008
:101EDC00CBE7C046F801002010B5034B0100186891
:101EEC0000F026F810BDC0461400002070B50F4E4F
:101EFC000D003168040011B900F034FE3060290087
:101F0C00200000F02FFE431C03D101256D42280058
:101F1C0070BD0323C51C9D43A842F8D0291A20008C
:101F2C0000F020FE0130F2D1EFE7C046F4010020B2
:101F3C00F7B50322CB1C9343083305001F000C2B71
:101F4C0034D20C27B94233D8384E280000F070F840
:101F5C0033681C00002C2FD139002800FFF7C6FF76
:101F6C000400431C5FD134680094009B002B4AD1C1
:101F7C00002C52D023682800E3180099019300F03C
:101F8C00F1FD019B834248D123682800FF1A3900D8
:101F9C00FFF7ACFF013040D02368DB1923603368B6
:101FAC005A68002A33D1009B336019E0002BC9DA40
:101FBC000C232B600020FEBD2168C91B20D40B29EB
:101FCC000AD9E2192760A34204D132606368116018
:101FDC00536005E05A60F9E76268A3420ED13260A3
:101FEC00280000F02DF8200007220B30231D904311
:101FFC00C21A9842DFD01B1AA350DCE75A60EFE7F5
:10200C0023006468A6E7009C63680093ADE71A00A0
:10201C005B68A342FBD10023DAE70C2328002B607A
:10202C0000F00EF8C6E70760DAE7C046F8010020BA
:10203C0010B50248FFF7FDFE10BDC046F0010020B0
:10204C0010B50248FFF7F6FE10BDC046F0010020A7
:10205C00F0B58E6885B01F000C000B6802900392DF
:10206C00BE4231D80C21625E40F280410A4229D036
:10207C00032021695B1A0193636943430198DD0FC7
:10208C00ED187B1C1B186D10AB4200D91D005205BE
:10209C0029D529000298FFF74BFF060000282DD008
:1020AC00019A2169FFF7C7FEA289194B1A408023B8
:1020BC001343A381019B2661F61826603E006561DF
:1020CC00ED1AA560BE4200D93E003200039920688B
:1020DC0000F014FD0020A3689B1BA36023689B19D0
:1020EC00236005B0F0BD2A00029800F056FD0600F2
:1020FC000028DFD121690298FFF7A6FE0C230120EE
:10210C00029A40421360A28934331343A381E8E757
:10211C007FFBFFFFF0B5A1B0039004921D008B89EB
:10212C000F001B060FD50B696BB94021FFF700FFA1
:10213C003860386128B90C23039A1360012040429F
:10214C00CFE040237B61002308AC636120336376CE
:10215C001033A3760795049E33780BB1252B46D10B
:10216C00049BF51A9E420BD02B003900049A03985D
:10217C00FFF76EFF013000D1AEE063695B1963615C
:10218C003378002B00D1A7E0012200235242626079
:10219C0004A95432521801362360E360A360137013
:1021AC00A36505223178544800F0ECFC751C00BB8B
:1021BC002268D30604D5532304A95B182021197077
:1021CC00130704D5532304A95B182B2119703378FA
:1021DC002A2B17D03500002140F20A0C0126E368A7
:1021EC002A78681C303A092A4ED989B917E0013689
:1021FC00B2E7414B2268C01A0123834013432E00DF
:10220C002360CEE7079B191D1B680791002B01DB90
:10221C000B9304E05B42E3600223134323602B78AF
:10222C002E2B0CD16B782A2B34D1079B02351A1D1F
:10223C001B680792002B01DA01235B4209932F4E96
:10224C0003223000297800F09DFC30B14023801B24
:10225C008340226801351343236029786B1C0622C6
:10226C0027480493217600F08DFC00283BD0254BA9
:10227C0033BB0722079B07339343083307936369E8
:10228C00059A9B18636166E761464B430500310074
:10229C009B18A5E7002340F20A0C1A000126013511
:1022AC0063602978681C3039092903D9002BC6D002
:1022BC000992C4E763465A43050033005218F0E70D
:1022CC0007AB00933A0021000F4B039800E000BFCE
:1022DC000590059B0133D2D1BB890D985B0600D5C7
:1022EC002CE721B0F0BD07AB00933A002100064B60
:1022FC00039800F0B7F9EBE79C370008A237000809
:10230C00A6370008000000005D200008936810B597
:10231C00013B9360002B04DA9469A34207DB0A2982
:10232C0005D01368581C10601970080010BDFFF719
:10233C0073FC0100F9E7F8B506000F001400D5187E
:10234C00AC4201D1002007E021783A003000FFF7C1
:10235C00DDFF0134431CF3D1F8BD0000F0B5A1B092
:10236C000D0017001E00039018B1036A0BB9FFF79C
:10237C00DDFA6B6EDB0705D4AB899B0502D4A86D27
:10238C00FFF757FDAB891B0701D52B6993B92900C2
:10239C000398FFF77FFC68B16B6EDB0703D5012058
:1023AC00404221B0F0BDAB899B05F8D4A86DFFF776
:1023BC0041FDF4E7002308AC6361203363761033EE
:1023CC00A37607963E0033780BB1252B46D1F31B31
:1023DC000593BE420BD03A0029000398FFF7ABFFE0
:1023EC00013000D1AEE06369059A9B1863613378C4
:1023FC00002B00D1A6E0012200235242626004A906
:10240C0054325218771C2360E360A3601370A365E9
:10241C0005223978574800F0B5FB7E1C00BB2268BA
:10242C00D30604D5532304A95B1820211970130774
:10243C0004D5532304A95B182B2119703B782A2B44
:10244C0017D03E00002140F20A0C0127E3683278D5
:10245C00701C303A092A4DD989B917E00136B2E718
:10246C00444B2268C01A0123834013433700236076
:10247C00CEE7079B191D1B680791002B01DB0B9303
:10248C0004E05B42E36002231343236033782E2B7A
:10249C000CD173782A2B33D1079B02361A1D1B687B
:1024AC000792002B01DA01235B420993324F03227E
:1024BC003800317800F066FB30B14023C01B8340FC
:1024CC002268013613432360317806222B48771C8F
:1024DC00217600F057FB002843D0294B33BB072251
:1024EC00079B07339343083307936369049A9B183C
:1024FC00636167E761464B43060039009B18A6E70A
:10250C00002340F20A0C1A0001270136636031786F
:10251C00701C3039092903D9002BC7D00992C5E7A3
:10252C0063465A4306003B005218F0E707AB009392
:10253C002A002100134B039800E000BF0490049B79
:10254C000133D2D16B6EDB0705D4AB899B0502D46A
:10255C00A86DFFF76FFCAB895B0600D51FE70D98E4
:10256C001FE707AB00932A002100064B039800F0ED
:10257C0079F8E3E79C370008A2370008A637000873
:10258C000000000043230008F7B5160001938A6889
:10259C000B690C000090934200DA130022003360A8
:1025AC00433212780AB10133336023689B0602D59B
:1025BC003368023333602268062315001D401A422B
:1025CC0027D0230043331B785A1E9341226892066E
:1025DC0030D4220001990098089D4332A84701305D
:1025EC0025D00622236800251340042B05D133681F
:1025FC00E568ED1AEB43DB171D40A3682269934293
:10260C0001DD9B1AED180026B54220D1002010E008
:10261C000135E36832689B1AAB42D2DD22000123FC
:10262C0001990098089F1932B8470130F0D1012068
:10263C004042FEBD3020E1184331087021005A1C85
:10264C0045310978A218433202331170C1E72200D8
:10265C00012301990098089F1A32B8470130E6D03F
:10266C000136D1E7F0B50E0089B0049203900593C2
:10267C000C00097E0E9A4336782907D8622909D8AE
:10268C00002900D1B7E0582900D1A0E0250042353F
:10269C00297022E0080063381528F7D8FDF710FDE3
:1026AC0016001F00F6FFF6FFF6FFF6FF1F00F6FF01
:1026BC00F6FFF6FFF6FF9E0034004300F6FFF6FF30
:1026CC00AF00F6FF3400F6FFF6FF47002500136855
:1026DC004235191D1B6811602B7001239CE0136897
:1026EC002068191D050609D51B681160002B02DA3C
:1026FC002D225B4232700A225B4832E01B6811606B
:10270C004006F3D51BB2F1E71068256808C82F0600
:10271C0002D46D0600D59BB21060082252486F2976
:10272C001BD00A2219E0202321680B432360782157
:10273C004E482300453319701568216808CD0F06E3
:10274C0002D44F0600D59BB21560CA0702D52022D1
:10275C000A432260002B3CD010222100002543317B
:10276C000D706168A160002908DB40F2040C67461B
:10277C0025681943BD432560350061B13500B3FBB5
:10278C00F2FC61465143591A415C013D2970190014
:10279C0063468A42F3D9082A09D12368DB0706D598
:1027AC00626823699A4202DC3023013D2B70761B50
:1027BC002661059B210000930398049B07AAFFF751
:1027CC00E3FE01302CD10120404209B0F0BD264877
:1027DC00AFE7202122688A432260BDE71368256891
:1027EC00181D616910601B682F0601D5196002E085
:1027FC006D06FBD51980002335002361D9E71368DA
:10280C00191D11601D6800212800626800F0BAF9DA
:10281C0008B1401B60606368236100233370C8E714
:10282C002A00236904990398059DA8470130CAD052
:10283C0023689B0715D4079BE0689842C5DA1800FB
:10284C00C3E72200012304990398059E1932B0476F
:10285C000130B8D00135E368079A9B1AAB42F0DC23
:10286C00E9E70025F7E7C046AD370008BE3700089A
:10287C00F7B50C228B5E05000C001A0753D44A687E
:10288C00002A02DC0A6C002A4BDDE76A002F48D0D4
:10289C00002241F200002E682A601A00216A0240D0
:1028AC00034230D0626DA3895B0705D56368D21AE9
:1028BC00636B0BB1236CD21A00232800E76A216AE0
:1028CC00B847A289431C06D129681D2944D8284B36
:1028DC00CB40DB0740D50023636023692360D2041F
:1028EC0004D5431C01D12B6803B96065616B2E6064
:1028FC00B9B123004433994202D02800FFF7A4FA5F
:10290C00002363630DE001232800B8470200431C39
:10291C00C9D12B68002BC6D01D2B01D0162B1AD178
:10292C002E6000201EE00E69002EFAD00F680E609B
:10293C00BA1B019200229B0700D14A69A260019B3D
:10294C00002BEEDDA36A32001F002800019B216AD8
:10295C00B847002807DCA2894023012013431BB28F
:10296C00A3814042FEBD019B36181B1A0193E6E77A
:10297C00010040200B6970B505000C0013B900254F
:10298C00280070BD18B1036A0BB9FEF7CFFF0C22FB
:10299C00A35E002BF3D0626ED20704D49B0502D445
:1029AC00A06DFFF746FA28002100FFF761FF636E68
:1029BC000500DB07E4D4A3899B05E1D4A06DFFF7E8
:1029CC0039FADDE770B50E001D000E23C95E140048
:1029DC0096B000290CDAB2898023110019401A42F2
:1029EC0014D140F2004300202960236016B070BD62
:1029FC006A4600F095F80028EDDB4FF200030199D0
:102A0C001940044BC9184B425941EAE700214023B5
:102A1C00E9E7C04600E0FFFFF0B502268B89050010
:102A2C000C0085B0334207D0230047332360236169
:102A3C000123636105B0F0BD03AB02AAFFF7C2FF2F
:102A4C00029F019039002800FFF772FA40B90C225E
:102A5C00A35E9A05EED4032293431E43A681E3E7BB
:102A6C008023A28920601343A381039B20616761AB
:102A7C005BB128000E23E15E00F064F828B103235B
:102A8C00A2899A43023B1343A381A389019A13435E
:102A9C00A381CFE770B506000D00140018B1036ACE
:102AAC000BB9FEF743FF636EDB0705D4A3899B05C7
:102ABC0002D4A06DFFF7BDF9A368013BA360002B06
:102ACC0005DAA269934212DBEBB20A2B0FD0236812
:102ADC005A1C22601D70EDB2636EDB0705D4A3890E
:102AEC009B0502D4A06DFFF7A5F9280070BD290045
:102AFC0022003000FFF790F80500EDE710B5884292
:102B0C0002D98B18984208D300239A4207D0CC5C88
:102B1C00C4540133F9E78B5C8354013AFBD210BDEA
:102B2C00002370B5064D0400080011002B6000F066
:102B3C0073F8431C02D12B6803B1236070BDC046EF
:102B4C00EC010020002370B5054D040008002B603B
:102B5C0000F06CF8431C02D12B6803B1236070BDEC
:102B6C00EC010020002370B5054D040008002B601B
:102B7C0000F078F8431C02D12B6803B1236070BDC0
:102B8C00EC010020C9B28218904201D1002070479C
:102B9C0003788B42FBD00130F6E7F7B506000C004A
:102BAC00150029B91100FFF7C3F904002000FEBD80
:102BBC001AB9FFF749F92C00F8E700F01BF80700E9
:102BCC00854202D84308AB42F0D329003000FFF70E
:102BDC00AFF9019008B9019CE8E72A00BD4200D981
:102BEC003A0021000198FFF726F921003000FFF789
:102BFC002BF9F0E70B1F1B68181F002B01DA0B5881
:102C0C00C018704740F2EC1358220120C2F20003A6
:102C1C0040421A607047C04640F2EC135822012023
:102C2C00C2F2000340421A607047C04640F2EC13F7
:102C3C005822C2F2000300201A60704740F2EC13D5
:102C4C0058220120C2F2000340421A607047C0466D
:102C5C0040F2EC1358220120C2F2000340421A60E9
:102C6C007047C04640F2FC12C2F20002030010682A
:102C7C0010B1C3181360704740F20020C2F200007C
:102C8C00F7E7C0469E2110B5C905041CFDF752FAA2
:102C9C0018B9201C00F024FC10BD9E21201CC90575
:102CAC0000F05AFA00F01CFC80231B069C46604482
:102CBC00F2E7C046F0B546464F46D646C0B547008B
:102CCC004502C30F3F0E98460E1C6D0A002F56D0BE
:102CDC00FF2F21D0802340F2000940F2000AED00C2
:102CEC00DB041D437F3F730074021B0E640AF60F56
:102CFC0003B3FF2B4AD080220020E400D2041443FB
:102D0C007F3B4246FF1A4B4672400F2B00D9AAE07C
:102D1C006E499B00CB589F46002D59D1730074020D
:102D2C001B0E40F20809FF2740F2020A640AF60F54
:102D3C00002BDED174BB0123424649467240194335
:102D4C000E2904D86248890041588F464246FF201C
:102D5C000024C0052043D2071043E0BCBA46B1465C
:102D6C00A846F0BD5346022BF0D0032B00D1A2E0B5
:102D7C0042462C00012B34D100200024E9E7D5B9C0
:102D8C0040F20409002740F2010AACE764B90223BF
:102D9C00FF3FD1E72000FDF7D7F9431F9C40762376
:102DAC005B421B1A0020ACE703234A461A439146A8
:102DBC000320FC33A5E72800FDF7C6F97627431F4F
:102DCC007F429D4040F2000940F2000A3F1A8AE718
:102DDC0040F20C09FF2740F2030A84E703286CD069
:102DEC00320038007F30002825DD630704D00F2324
:102DFC002340042B00D00434230103D53800354B79
:102E0C0080301C40FE28A2DCA401640AC0B2A0E7FA
:102E1C0080240022FF20E4039BE78023DB031D4278
:102E2C0001D01C424BD08024E4032C436402424664
:102E3C00FF20640A8DE701231B1A1B2B9CDC21004D
:102E4C009E37D940BC400B00611E8C41234359076F
:102E5C0004D00F211940042900D00433590126D580
:102E6C000120002475E76D016001854213D21B23FC
:102E7C000024013F0126290064006D00002901DBBC
:102E8C00A84201D82D1A3443013B002BF3D16B1E01
:102E9C009D412C43A5E71A2301242D1AEAE7981E1D
:102EAC0043425841404232000024C0B251E79B01DA
:102EBC0000205C0A4DE746462C008023DB031C43B4
:102ECC0064023200FF20640A43E7C046D037000892
:102EDC0010380008FFFFFFF7F0B54F464646D646C0
:102EEC00C0B546004502360E0F1C6D0AC40F002EED
:102EFC0000D1C4E0FF2E79D0802340F2000940F2CB
:102F0C00000AED00DB041D437F3E7B025B0A984602
:102F1C007B001B0EFF0F002B78D0FF2B00D195E010
:102F2C0042468021D200C9041143884600217F3BD0
:102F3C00F6184B46721C0A2B74DC4B467C40022B59
:102F4C0000DCA6E048460123834040F23050184292
:102F5C0068D140F24020184200D0ECE0B938FF387C
:102F6C00184200D0DAE04FF6FF714746280C434672
:102F7C000D4039400F001B0C6F4341435D435843D8
:102F8C006D183B0C5B19994203D9802149028C4680
:102F9C0060444FF6FF7519043D4049198D016F1EB1
:102FAC00BD411B0C890E1B180D439B011D431B01BE
:102FBC0000D4C5E0012369081D400D4310007F308B
:102FCC00002800DC93E06B0704D00F232B40042B6C
:102FDC0000D004352B0103D5803210005D4B1D4011
:102FEC00FE2853DCAB015B0AC0B226E0002D00D0FA
:102FFC0077E07B025B0A98467B001B0E40F20809C7
:10300C00FF2640F2020AFF0F002B86D14346002B0D
:10301C0055D14A4601331A4391464B460121721C45
:10302C000A2B8ADD5346022B30D0032B00D17BE0D8
:10303C005346012BC2D100200023C0051843E407DE
:10304C002043E0BCBA46B146A846F0BD3300424628
:10305C00FF33FAB3032249461143721C8946FF32EF
:10306C000A2973DD0F295DD18023DB031D425BD060
:10307C0042461A4258D13C00FF201343DDE78DB97C
:10308C0040F20409002640F2010A3EE7FF2000232B
:10309C00D3E7013B012B00D965E70229F6D0454661
:1030AC008A46C5E72800FDF74FF87626431F76427F
:1030BC009D4040F2000940F2000A361A25E74046CE
:1030CC00FDF742F84246431F9A40361A90460021BB
:1030DC00763E2EE749460232114389461E000221F4
:1030EC0027E740F20C09FF2640F2030A0DE7012303
:1030FC001B1A1B2B9FDC9E3229009540D9406A1E5F
:10310C0095410D436B0704D00F232B40042B00D0AB
:10311C0004356B0116D5012000238EE73C00454693
:10312C008A467FE73C0045468023DB032B435B024A
:10313C00FF205B0A81E780230024FF20DB037CE770
:10314C0032003BE7AB0100205B0A76E71E0003214F
:10315C007C40F7E6FFFFFFF7F0B546464F46D646F4
:10316C0043025B0AC0B59C461F00DE004B025A0AA4
:10317C00904645004A002D0EC40F120EC90F9B0934
:10318C00FF2A25D001204140A81A8C420FD00028DC
:10319C0000DC8AE192BB002B00D19CE0421E01288E
:1031AC0000D14FE1FF2800D19BE010002CE000285B
:1031BC0000DC87E1002A00D182E0FF2D00D190E0F5
:1031CC008022D20413431B2800DCEAE001363FE0E6
:1031DC002800FF388246002B54D140F201094846A2
:1031EC0041408C4200D1C4E05046002800D187E019
:1031FC000C00002D4CD0FF2000273AE0FF2D00D111
:10320C006FE08022D204134301221B2807DC20210B
:10321C00091A1A008B40C240591E8B411A43B61A28
:10322C0073016AD5B601B7093800FCF78DFF053874
:10323C008740854200DD7EE020223B00401B0130B0
:10324C00121A3E009340C6405A1E934100251E435D
:10325C00730704D00F233340042B00D004367301C2
:10326C003AD5681CFE2DC6D09B4BC0B233409B0197
:10327C005F0AC0053843E4072043E0BCBA46B146B8
:10328C00A846F0BD8C4264D0D0B3002D00D0A3E092
:10329C00FF20F6B1471E012800D1E1E00C00FF2809
:1032AC0000D1CDE001211B2F07DC2020C01B3100F9
:1032BC008640F940701E8641314315005E1AAFE717
:1032CC004BB1421E012800D1A0E0FF2809D010000C
:1032DC0079E70C001E000500F3089C46FF2D00D07A
:1032EC009BE06346002B00D185E780276346FF03F4
:1032FC001F437F02FF207F0ABBE77307AAD1EBE7CE
:10330C00FE206A1C10421AD1002D77D1002E00D15C
:10331C00AAE00020002BACD08022F71AD20417426E
:10332C0000D1BBE001249B1B0C4013429FD06A4A86
:10333C00013013409BE7684E2D1A3E4088E7F71A80
:10334C007A0157D4002F00D06EE70024002000270C
:10335C008FE780B1002D73D1FF20002EBAD0411E13
:10336C00012853D0FF286BD01B296EDD15005E1C85
:10337C006EE7514659BBFE216A1C114233D1002D18
:10338C0050D1002E00D186E00020002B00D170E738
:10339C00F318DF087F027F0A5B0100D469E7012084
:1033AC0067E72021091A1A008B40C240591E8B4135
:1033BC001343F6187301A0D50135FF2D00D11AE780
:1033CC000123464A3340760816401E4340E7002D41
:1033DC0000D010E7FF20C0E70C00C44681E7FE21B7
:1033EC006A1C0A42CDD0FF2A00D104E7F61815005A
:1033FC0076082DE701249F1B0C4015E7E6BB002B3C
:10340C0045D180270024FF20FF0332E7F618022560
:10341C007301D5D4F3089C46012563465F027F0AED
:10342C00E8B226E766B1002B00D15EE78023DB0310
:10343C009C4500D259E7984500D356E7C44654E75B
:10344C00C4464EE70125F61AEAE630002025C840AE
:10345C00691A8E40711E8E4106431500F618A9E7B5
:10346C000C0001259E1BDBE6002B00D16DE701242F
:10347C00474600200C40FCE6002B00D135E78023AA
:10348C00DB039C4500D230E7984500D32DE701249F
:10349C00C4460C4029E747460020EAE617B1BF01B5
:1034AC007F0AE6E600240027E3E6002800D127E7A0
:1034BC00571B3800002D00D1EBE68020C0040C0017
:1034CC000643EFE600288AD0511B0DB9080044E7EB
:1034DC008020C004064347E7FFFFFFFBFFFFFF7D93
:1034EC0041024200C30F490A0020120E7E2A03DD5E
:1034FC009D2A02DD094A9818704780200004014378
:10350C00952A07DC9620821AD1404842002BF3D131
:10351C000800F1E7963A9140F7E7C046FFFFFF7FBE
:10352C0070B5040070B1FCF70FFE03009E20C01AAA
:10353C0096280CDC082B2DD0083B9C406402640AB6
:10354C00C0B201E000200024C005204370BD9928C2
:10355C0014DC5A1F9440220010490A40650709D018
:10356C000F252C40042C05D00432540102D59F2089
:10357C000A40C01A9201540AC0B2E5E71A002100B1
:10358C001B3291400A00511E8A410521C91ACC40B8
:10359C001443E0E764029620640AD5E7FFFFFFFBC3
:1035AC0070B542004E024C0045026D0A120EC30F5C
:1035BC00760A240EC90FFF2A0FD0FF2C0BD0012046
:1035CC00A24209D1B54207D18B420FD022B92800B3
:1035DC00431E984100E0012070BD0120FF2CFBD15F
:1035EC003543002DF8D14B401800F5E70020F3E7E8
:1035FC0030B5420044024D02C30F4800640A120E5B
:10360C006D0A000EC90FFF2A12D0FF2807D0B2B9DD
:10361C0038B90DB3002C2AD14800013830BD1DBB80
:10362C000AB9002CF8D08B4205D158000138F5E7C7
:10363C00D4B9FF2813D001205B421843EEE70028D1
:10364C00F9D08B42F7D18242F5DCEEDBAC42F2D8FA
:10365C000020AC42E2D2E8E7002CDFD0EBE71DB94A
:10366C008B42E8D10020D9E702204042D6E78B42BA
:10367C00ECD0E0E730B5420044024D02C30F4800E5
:10368C00640A120E6D0A000EC90FFF2A12D0FF2811
:10369C0006D0AAB930B915B344BB480001380EE0C6
:1036AC0065B90AB9002CF8D08B4215D001205B42C9
:1036BC00184304E014B9FF28F8D19DB1022030BDA5
:1036CC000028F3D08B42F1D18242EFDC04DBAC4218
:1036DC00ECD80020AC42F2D258000138EFE7002CB5
:1036EC00EDD0E3E700208B42E9D0DFE78B42EED050
:1036FC00DCE7C046F8B5C046F8BC08BC9E4670472F
:0C370C00F8B5C046F8BC08BC9E467047EB
:103718000000000000000000010203040607080979
:1037280000000000010203042563256325630000EF
:103738002563256300000000256325632563256351
:103748002563256300000000256325632563256341
:103758002563256325630000D60700080C080008C8
:103768002E080008D207000850080008D2070008F1
:10377800D2070008D2070008B20700086C13000837
:1037880006130008AA13000808130008B01300085D
:1037980070130008232D302B2000686C4C006566E0
:1037A800674546470030313233343536373839418A
:1037B80042434445460030313233343536373839A0
:1037C8006162636465660000722E00085A2D000865
:1037D800842D0008E82D0008842D00081C2E000800
:1037E800842D0008E82D00085A2D00085A2D0008DD
:1037F8001C2E0008E82D0008702D0008702D000808
:10380800702D0008262E00085A2D00085A2D000891
:10381800842D0008AA2E0008842D00081C2E0008FC
:10382800842D0008AA2E00085A2D00085A2D0008D9
:103838001C2E0008AA2E0008702D0008702D000804
:04384800702D0008D7
:04384C00110200085D
:04385000E10100088A
:10385400B5F0040000A24A040000000003000000C8
:10386400B00000201800002000000000B00000207C
:10387400180100208001002000000000000000006A
:103884000000000000000000000000000000000034
:103894000000000000000000000000000000000024
:1038A4000000000000000000000000000000000014
:0438B4000000000010
:04000005080017C513
:00000001FF
